:100000000C942A000C9445000C9445000C94450077
:100010000C9445000C9445000C9445000C9447004A
:100020000C9445000C9445000C9445000C9445003C
:100030000C9445000C9445000C9445000C9445002C
:100040000C9445000C9445000C9445000C9445001C
:100050000C94450011241FBECFE5D8E0DEBFCDBF14
:1000600010E0A0E6B0E0EAE2F2E002C005900D92F6
:10007000A436B107D9F710E0A4E6B0E001C01D92A4
:10008000A536B107E1F70C949C000C9400001F9278
:100090000F920FB60F9211242F933F938F939F933C
:1000A00080916400813069F0813028F0823059F00D
:1000B0008330D1F412C0AF98209162003091630078
:1000C00007C0AE9A0BC0AE982091600030916100DD
:1000D00080E098E2821B930B05C0AF9A809160008C
:1000E000909161009BBD8ABD809164008F5F809379
:1000F0006400809164008370809364009F918F916D
:100100003F912F910F900FBE0F901F901895A69AB8
:10011000AE98A79AAF9885B38F6085BB1FBC1DBCF6
:100120001CBC80E098E29BBD8ABD89B7806189BF15
:100130008AE08EBD78940895CFE5D8E0DEBFCDBFCC
:100140000E94870040E058E020E034E0E0E2FEE476
:1001500083B399278F7090708B30910521F18C308B
:10016000910524F4079709F05CC007C08D30910514
:1001700079F10E9709F055C040C0809160009091D0
:10018000610001969093610080936000809160000F
:10019000909161008150984008F443C050936100F1
:1001A000409360003EC08091600090916100019793
:1001B0009093610080936000809160009091610055
:1001C0008050944070F5309361002093600029C006
:1001D00080916200909163000196909363008093F8
:1001E0006200809162009091630081509840C8F055
:1001F000509363004093620014C08091620090911C
:100200006300019790936300809362008091620085
:10021000909163008050944020F4309363002093C9
:0A0220006200CF010197F1F793CFC0
:04022A0000060006C4
:00000001FF
